:020000040000FA
:020000000528D1
:08000800472883018B018501EB
:100010000730990083162F30850070308F008830AC
:100020008100831281018B128B17C20142182D2887
:10003000851A162805080F3A0F3903191030C30026
:100040003C30C40042140516383081002430C00012
:100050005F30C1008B163720162843080319322859
:10006000851A16288B120512C20137201628143063
:10007000C500FA30C6002730C70000000000C70BDB
:100080003D280000C60B3B28C50B39280800F000AE
:100090000308F10083120B1D64280B113830810016
:1000A0000130C1020319582803186428C0026428CB
:1000B000C008031D64282430C0005F30C100C40B99
:1000C00064283C30C400C30371088300F00E700E36
:0200D000090025
:02400E00C43CB0
:00000001FF
